:020000040800F2
:1000000000280020050E0008490E0008490E0008CF
:10001000490E0008490E0008490E000800000000C3
:10002000000000000000000000000000490E000871
:10003000490E000800000000490E0008D10D00081C
:10004000490E0008490E0008490E0008490E000834
:10005000490E0008490E0008490E0008490E000824
:10006000490E0008490E0008490E0008490E000814
:10007000490E0008490E0008490E0008490E000804
:10008000490E0008490E0008490E0008490E0008F4
:10009000490E0008490E0008490E0008490E0008E4
:1000A000490E0008490E0008490E0008490E0008D4
:1000B000490E0008490E000800000000490E000823
:1000C000490E00080000000000000000490E000872
:1000D00000000000490E0008490E00080000000062
:1000E000490E0008490E0008490E000800000000F3
:1000F0000000000000000000000000000000000000
:0C01000000000000000000005FF808F1A3
:10010C0080B483B000AF03463960FB7197F90730B8
:10011C00002B0BDA0D49FB7903F00F03043B3A6813
:10012C00D2B21201D2B20B441A7609E0084997F9FF
:10013C0007303A68D2B21201D2B20B4483F80023D2
:10014C0000BF0C37BD4680BC704700BF00ED00E01F
:10015C0000E100E080B582B000AF78607B68B3F15D
:10016C00807F01D3012311E00A4A7B6823F07F438F
:10017C00013B53600F214FF0FF30FFF7C1FF054BE0
:10018C0000229A60034B07221A6000231846083796
:10019C00BD4680BD10E000E080B500AF154A154BA0
:1001AC001B6843F0010313601249124B5A68124B3F
:1001BC0013404B600F4A0F4B1B6823F0847323F4DE
:1001CC00803313600B4A0B4B1B6823F480231360A2
:1001DC00084A084B5B6823F4FE035360054B4FF44D
:1001EC001F029A6000F078F8044B4FF000629A609E
:1001FC0000BF80BD001002400000FFF800ED00E0E1
:10020C0080B485B000AF0023FB600023BB600023EB
:10021C007B602C4B5B6803F00C03FB60FB68042BCE
:10022C0007D0082B09D0002B33D1274B274A1A6053
:10023C0033E0254B254A1A602FE0224B5B6803F410
:10024C007013BB601F4B5B6803F480337B60BB682F
:10025C009B0C0233BB607B68002B06D1BB681C4A2D
:10026C0002FB03F3184A136017E0164B5B6803F4A8
:10027C000033002B06D0BB68154A02FB03F3124A6D
:10028C0013600AE0BB68114A02FB03F30E4A1360C9
:10029C0003E00D4B0D4A1A6000BF0A4B5B6803F07C
:1002AC00F0031B090B4AD35CDBB2FB60064B1A68EC
:1002BC00FB6822FA03F3044A136000BF1437BD46EF
:1002CC0080BC7047001002400000002000127A0031
:1002DC0000093D000400002080B500AF00F002F8DA
:1002EC0000BF80BD80B483B000AF00237B600023CF
:1002FC003B603A4A394B1B6843F480331360374BED
:10030C001B6803F400333B607B6801337B603B6804
:10031C00002B03D17B68B3F5A06FF0D12F4B1B687A
:10032C0003F40033002B02D001233B6001E00023D7
:10033C003B603B68012B4BD1294A294B1B6843F08E
:10034C0010031360264A264B1B6823F0030313602B
:10035C00234A234B1B6843F0020313601F4A1F4BB5
:10036C005B6853601D4A1D4B5B6853601B4A1B4BFB
:10037C005B6843F480635360184A184B5B6823F442
:10038C007C135360154A154B5B6843F4E8135360B8
:10039C00124A124B1B6843F08073136000BF0F4B63
:1003AC001B6803F00073002BF9D00C4A0B4B5B68F5
:1003BC0023F003035360094A084B5B6843F00203C4
:1003CC00536000BF054B5B6803F00C03082BF9D19D
:1003DC0000BF0C37BD4680BC704700BF0010024008
:1003EC000020024080B483B000AF78600B46FB70F5
:1003FC00FB78002B06D07B689B6843F001027B687E
:10040C009A6005E07B689B6823F001027B689A6028
:10041C0000BF0C37BD4680BC704700BF80B485B0B0
:10042C0000AF78600B467B800023FB737B681B89D5
:10043C009AB27B8813409BB2002B02D00123FB7332
:10044C0001E00023FB73FB7B18461437BD4680BCD0
:10045C00704700BF80B483B000AF78600B467B80E0
:10046C007B687A889A8100BF0C37BD4680BC704788
:10047C0080B483B000AF78607B689B6843F008025F
:10048C007B689A6000BF0C37BD4680BC704700BFCC
:10049C0080B485B000AF78600023FB737B689B68E9
:1004AC0003F00803002B02D00123FB7301E00023AF
:1004BC00FB73FB7B18461437BD4680BC704700BFEE
:1004CC0080B483B000AF78607B689B6843F0040213
:1004DC007B689A6000BF0C37BD4680BC704700BF7C
:1004EC0080B485B000AF78600023FB737B689B6899
:1004FC0003F00403002B02D00123FB7301E0002363
:10050C00FB73FB7B18461437BD4680BC704700BF9D
:10051C0080B483B000AF78600B46FB70FB78002B87
:10052C0006D07B689B6843F4A0027B689A6005E068
:10053C007B689B6823F4A0027B689A6000BF0C3731
:10054C00BD4680BC704700BF80B483B000AF7860FC
:10055C007B689B899BB218460C37BD4680BC7047A4
:10056C0080B582B000AF0346FB7100BF02210E487C
:10057C00FFF754FF0346002BF8D0FB799BB21946CA
:10058C000948FFF767FF00BF01210748FFF746FF47
:10059C000346002BF8D00448FFF7D6FF0346DBB226
:1005AC0018460837BD4680BD0030014080B489B084
:1005BC0000AF786039600023FB6100233B610023AE
:1005CC00BB610023FB6000237B610023BB603B68A5
:1005DC00DB7803F00F03FB613B68DB7803F010035F
:1005EC00002B05D03B689B781A46FB691343FB61D3
:1005FC003B681B88DBB2002B44D07B681B687B619B
:10060C000023BB6138E00122BB6902FA03F3FB60F3
:10061C003B681B881A46FB6813403B613A69FB68D0
:10062C009A4226D1BB699B00FB600F22FB6802FA41
:10063C0003F3BB60BB68DB437A6913407B61FA69E7
:10064C00FB6802FA03F37A6913437B613B68DB783E
:10065C00282B05D10122BB699A407B685A6108E0BE
:10066C003B68DB78482B04D10122BB699A407B683C
:10067C001A61BB690133BB61BB69072BC3D97B68AA
:10068C007A691A603B681B88FF2B46D97B685B68CC
:10069C007B610023BB613AE0BB690833012202FA9B
:1006AC0003F3FB603B681B881A46FB6813403B61F5
:1006BC003A69FB689A4227D1BB699B00FB600F2209
:1006CC00FB6802FA03F3BB60BB68DB437A69134037
:1006DC007B61FA69FB6802FA03F37A6913437B6165
:1006EC003B68DB78282B05D1BB69083301229A4083
:1006FC007B685A613B68DB78482B05D1BB690833B2
:10070C0001229A407B681A61BB690133BB61BB69EA
:10071C00072BC1D97B687A695A6000BF2437BD4664
:10072C0080BC704780B485B000AF7860396000231E
:10073C00FB817B681B88FB81FB8903F44153FB81A4
:10074C003B681A883B685B8813439AB23B689B886A
:10075C0013439AB23B68DB8813439AB23B681B89FC
:10076C0013439AB23B685B8913439AB23B689B89EB
:10077C0013439AB23B68DB8913439AB2FB89134348
:10078C00FB817B68FA891A807B689B8B9BB223F474
:10079C0000639AB27B689A833B681A8A7B681A82D8
:1007AC0000BF1437BD4680BC704700BF80B483B017
:1007BC0000AF78600B46FB70FB78002B08D07B6891
:1007CC001B889BB243F040039AB27B681A8007E007
:1007DC007B681B889BB223F040039AB27B681A801B
:1007EC0000BF0C37BD4680BC704700BF80B483B0DF
:1007FC0000AF78600B467B807A887B681A6100BFFB
:10080C000C37BD4680BC704780B483B000AF7860B5
:10081C000B46FB70FB78002B06D00949084B9A69F4
:10082C007B6813438B6106E00549054B9A697B682D
:10083C00DB4313408B6100BF0C37BD4680BC704757
:10084C000010024080B483B000AF78600B467B8010
:10085C007A887B685A6100BF0C37BD4680BC7047F4
:10086C0080B485B000AF786039600023FB60002352
:10087C00FB727B685B68FB60FB6803F44153FB60B5
:10088C003B681A683B681B791B021343FA681343D5
:10089C00FB607B68FA685A607B689B68FB60FA684F
:1008AC00164B1340FB603B68DA683B689B681A4345
:1008BC003B685B795B001343FA681343FB607B680E
:1008CC00FA689A607B68DB6AFB60FB6823F4700350
:1008DC00FB603B681B7C013BDAB2FB7A1343FB7277
:1008EC00FB7A1B05FA681343FB607B68FA68DA62D3
:1008FC0000BF1437BD4680BC704700BFFDF7F1FF49
:10090C0080B586B000AF01210420FFF77DFF0121E7
:10091C004FF48050FFF778FFE023BB820323BB75B5
:10092C001823FB7507F1140319461748FFF73EFE11
:10093C001023BB821023FB7507F1140319461248D0
:10094C00FFF734FE00233B804FF482737B8000233F
:10095C00BB800223FB8001233B814FF400737B811E
:10096C000823BB810023FB8107233B823B461946AE
:10097C000648FFF7D7FE01210448FFF717FF00BF19
:10098C001837BD4680BD00BF000801400030014053
:10099C0080B500AF10211848FFF754FF95220021B5
:1009AC00002000F02BF8012000F05EF80346002B2D
:1009BC0001D0FF231DE010210F48FFF717FFFF2088
:1009CC00FFF7CEFD10210C48FFF73CFFFF22002162
:1009DC00012000F013F8002000F046F80346002B2D
:1009EC00E9D110210448FFF701FFFF20FFF7B8FD04
:1009FC000023184680BD00BF0008014080B586B0BA
:100A0C0000AF03463960FB711346BB7100237B6159
:100A1C00FB7943F04003DBB23B733B681B0EDBB24C
:100A2C007B733B681B0CDBB2BB733B681B0ADBB2F2
:100A3C00FB733B68DBB23B74BB797B7400237B613B
:100A4C000AE007F10C027B6913441B781846FFF788
:100A5C0087FD7B6901337B617B69052BF1D900BF75
:100A6C001837BD4680BD00BF80B584B000AF0346CB
:100A7C00FB7140F6FF73FB6002E0FB68013BFB601F
:100A8C0000F012F803461A46FB79934202D0FB6839
:100A9C00002BF2D1FB68002B01D1FF2300E00023D7
:100AAC0018461037BD4680BD80B582B000AF00231C
:100ABC00FB7100BF02210E48FFF7B0FC0346002B70
:100ACC00F8D0FF210A48FFF7C5FC00BF01210848F8
:100ADC00FFF7A4FC0346002BF8D00548FFF734FDC4
:100AEC000346FB71FB7918460837BD4680BD00BF35
:100AFC000030014080B582B000AF00237B601EE067
:100B0C00FFF7D2FF0346FB70FB7803F01F03FB706B
:100B1C00FB780B2B06D00D2B06D0052B06D105230D
:100B2C00BB7006E00B2316E00D2314E0FF23BB7013
:100B3C0000BFBB78052B06D07B6801337B607B68DC
:100B4C00402BDDD900E000BF00BFFFF7ADFF03462F
:100B5C00002BFAD0FB7818460837BD4680BD00BF85
:100B6C0080B582B000AF00237B60FFF7C9FE102177
:100B7C000A48FFF73BFE00237B6005E0FF20FFF7F0
:100B8C00EFFC7B6801337B607B68092BF6D9FFF7A0
:100B9C00FFFE034618460837BD4680BD00080140DD
:100BAC0080B500AF094B1B88002B01D100230AE054
:100BBC00FFF7D6FF03469AB2044B1A80034B1B88EF
:100BCC00002BF5D10123184680BD00BF1800002072
:100BDC0080B500AF00BFFFF7E3FF0346002BFAD14F
:100BEC0000BF80BD80B483B000AF78607B68DB6CE5
:100BFC009BB218460C37BD4680BC704780B584B09C
:100C0C0000AF78603B4B1A783B4B1A70394B002283
:100C1C001A700023FB60FF23FB7210213748FFF78B
:100C2C0011FEFF2279681820FFF7E8FE0020FFF77D
:100C3C001BFF0346002B4ED1FF20FFF791FCFE203B
:100C4C00FFF78EFC2C4B1B78012B1AD10023FB6079
:100C5C0014E02B4AFB6832F81330DBB21846FFF76E
:100C6C007FFC274AFB6832F813301B0A9BB2DBB2BD
:100C7C001846FFF775FCFB680133FB60FB68FF2B24
:100C8C00E7D91D4B1B78022B1AD10023FB6014E013
:100C9C001C4AFB6832F81330DBB21846FFF760FCD5
:100CAC00184AFB6832F813301B0A9BB2DBB21846A9
:100CBC00FFF756FCFB680133FB60FB68FF2BE7D9A1
:100CCC00FFF7F2FEFFF7F0FEFFF714FF0346052BCC
:100CDC0001D10023FB7210210848FFF787FDFF208C
:100CEC00FFF73EFC044B00221A70FB7A18461037B3
:100CFC00BD4680BD300600201B00002000080140CE
:100D0C00300200203004002080B586B000AF0121F5
:100D1C004FF40070FFF778FD01233B800023FB703C
:100D2C000223BB703B4619461A48FFF73FFC0023D1
:100D3C007B6001233B7201237B724FF46023FB60C9
:100D4C0000233B6100233B753B1D19461248FFF7FE
:100D5C0087FD01211048FFF745FB0F48FFF788FB83
:100D6C0000BF0D48FFF794FB0346002BF9D10A484E
:100D7C00FFF7A6FB00BF0848FFF7B2FB0346002BAA
:100D8C00F9D101210448FFF7C3FB00BF1837BD465A
:100D9C0080BD00BF000801400024014080B500AFB9
:100DAC00FFF72EFA054B1B68054AA2FB0323DB0851
:100DBC001846FFF7CFF9FFF7A7FFFEE7000000206A
:100DCC00CDCCCCCC80B500AF0448FFF70BFF03466D
:100DDC001A46034B1A8000BF80BD00BF002401409F
:100DEC002C0200204C0E0008000000201C000020EB
:100DFC001C00002038060020002103E00A4B5B5841
:100E0C004350043109480A4B42189A42F6D3094A16
:100E1C0002E0002342F8043B074B9A42F9D3FFF758
:100E2C00BBF9FFF7BBFF70474C0E00080000002019
:100E3C001C0000201C00002038060020FEE70000EB
:100E4C0000A24A040000000000000000010203049C
:0C0E5C00060708090A000000FFFF010261
:0400000508000E05DC
:00000001FF
